:100000000C9462000C948A000C948A000C948A0070
:100010000C948A000C948A000C948A000C948A0038
:100020000C948A000C948A000C948A000C948A0028
:100030000C948A000C948A000C948A000C948A0018
:100040000C94A5030C948A000C9473030C944D0338
:100050000C948A000C948A000C948A000C948A00F8
:100060000C948A000C948A000000000024002700F1
:100070002A0000000000250028002B0000000008D6
:10008000000201000003040700000000000000005F
:1000900000000000230026002900040404040404D6
:1000A0000404020202020202030303030303010227
:1000B00004081020408001020408102001020408F6
:1000C0001020EF0311241FBECFEFD8E0DEBFCDBF5D
:1000D00011E0A0E0B1E0E6E7F1E102C005900D9289
:1000E000AA32B107D9F723E0AAE2B1E001C01D921C
:1000F000A038B207E1F710E0C2E6D0E004C02197D3
:10010000FE010E94B308C136D107C9F70E947E04E0
:100110000C94B9080C940000AF92BF92CF92DF927A
:10012000EF92FF920F931F93CF93DF936C017B01AC
:100130008B01040F151FEB015E01AE18BF08C0173D
:10014000D10759F06991D601ED91FC910190F081B0
:10015000E02DC6010995892B79F7C501DF91CF9173
:100160001F910F91FF90EF90DF90CF90BF90AF90D5
:100170000895FC01538D448D252F30E0842F90E0AD
:10018000821B930B541710F0CF9608950197089592
:10019000FC01918D828D981761F0A28DAE0FBF2F5B
:1001A000B11D5D968C91928D9F5F9F73928F90E0B1
:1001B00008958FEF9FEF0895FC01918D828D981720
:1001C00031F0828DE80FF11D858D90E008958FEF5D
:1001D0009FEF0895FC01918D228D892F90E0805C26
:1001E0009F4F821B91098F73992708958FE391E0A8
:1001F0000E94EA0021E0892B09F420E0822F089573
:1002000080E090E0892B29F00E94F60081110C9487
:1002100000000895FC01A48DA80FB92FB11DA35AA9
:10022000BF4F2C91848D90E001968F739927848F16
:10023000A689B7892C93A089B1898C918370806439
:100240008C93938D848D981306C00288F389E02DDA
:1002500080818F7D80830895EF92FF920F931F938B
:10026000CF93DF93EC0181E0888F9B8D8C8D981369
:100270001AC0E889F989808185FF15C09FB7F89475
:10028000EE89FF896083E889F989808183708064C1
:1002900080839FBF81E090E0DF91CF911F910F910C
:1002A000FF90EF900895F62E0B8D10E00F5F1F4F1B
:1002B0000F731127E02E8C8D8E110CC00FB607FC2A
:1002C000FACFE889F989808185FFF5CFCE010E94B8
:1002D0000A01F1CFEB8DEC0FFD2FF11DE35AFF4F1B
:1002E000F0829FB7F8940B8FEA89FB898081806246
:1002F000CFCFCF93DF93EC01888D8823B9F0AA8903
:10030000BB89E889F9898C9185FD03C0808186FDD0
:100310000DC00FB607FCF7CF8C9185FFF2CF80811F
:1003200085FFEDCFCE010E940A01E9CFDF91CF9189
:10033000089590E0FC01E458FF4F2491FC01E25540
:10034000FF4F3491FC01E656FF4FE491EE23C9F0D4
:10035000222339F0233001F1A8F4213019F12230A1
:1003600029F1F0E0EE0FFF1FEE58FF4FA591B49179
:100370008FB7F894EC91611126C030953E233C93E1
:100380008FBF08952730A9F02830C9F0243049F7ED
:10039000809180008F7D03C0809180008F77809353
:1003A0008000DFCF84B58F7784BDDBCF84B58F7DB0
:1003B000FBCF8091B0008F778093B000D2CF809137
:1003C000B0008F7DF9CF3E2BDACFCF93DF9390E053
:1003D000FC01E255FF4F249186569F4FFC0184910A
:1003E0008823D1F090E0880F991FFC01E859FF4F56
:1003F000A591B491FC01EE58FF4FC591D4916111C4
:100400000EC09FB7F8948C91E22FE0958E238C93C9
:100410002881E223E8839FBFDF91CF9108958FB7B2
:10042000F894EC91E22BEC938FBFF6CF3FB7F894A2
:1004300080912F0190913001A0913101B091320152
:1004400026B5A89B05C02F3F19F00196A11DB11D2F
:100450003FBFBA2FA92F982F8827BC01CD01620F6B
:10046000711D811D911D43E0660F771F881F991F25
:100470004A95D1F708958F929F92AF92BF92CF92F3
:10048000DF92EF92FF924B015C010E9416026B011A
:100490007C010E9416026C197D098E099F09683E35
:1004A000734081059105A8F321E0821A9108A10803
:1004B000B10888EEC80E83E0D81EE11CF11C81143F
:1004C0009104A104B10429F7FF90EF90DF90CF9041
:1004D000BF90AF909F908F9008952FB7F894609140
:1004E0002B0170912C0180912D0190912E012FBF35
:1004F00008951F93CF93DF93EC01162F81E090E0D6
:100500009983888386E391E09F838E8380EF9AEBC3
:10051000A4E0B0E088879987AA87BB8780E29EE441
:10052000A0E0B0E08C879D87AE87BF8761E080E167
:100530000E94E50160E0812F0E94E50160E080E11A
:100540000E949901EEEBF0E0E491E88FEAEAF0E036
:10055000E491F0E0EE0FFF1FE057FF4F859194917B
:100560009A8F898F612F70E0FB01E255FF4FE49174
:10057000EB8FFB01E656FF4FE491F0E0EE0FFF1F1B
:10058000E057FF4F859194919D8F8C8F8FEF9FEF58
:10059000AFEFBFE08A839B83AC83BD830E946D0273
:1005A000688B798B8A8B9B8BDF91CF911F910895FC
:1005B000FC0101900020E9F73197AF01481B590B6E
:1005C000BC018FE391E00C948C008F929F92AF92CC
:1005D000BF92CF92DF92EF92FF920F931F93CF9330
:1005E000DF93CDB7DEB7A1970FB6F894DEBF0FBE8D
:1005F000CDBF8BE191E00E94D80285E291E00E949C
:10060000D80207E311E08EE3E82E81E0F82E9AE0AD
:10061000892E912CA12CB12CF80121918F0130E071
:1006200050E040E019A26E01F1E2CF0ED11CCA01E8
:10063000B901A50194010E949108605DF6016293E1
:100640006F01211531054105510589F7309719F0E2
:10065000CF010E94D80288E291E00E94D802E01601
:10066000F106D1F689E291E00E94D80285E291E09C
:100670000E94D802A1960FB6F894DEBF0FBECDBF80
:10068000DF91CF911F910F91FF90EF90DF90CF906E
:10069000BF90AF909F908F9008951F920F920FB6CA
:1006A0000F9211242F933F934F935F936F937F93F8
:1006B0008F939F93AF93BF93EF93FF938FE391E05B
:1006C0000E940A01FF91EF91BF91AF919F918F918D
:1006D0007F916F915F914F913F912F910F900FBE3E
:1006E0000F901F9018951F920F920FB60F92112422
:1006F0002F938F939F93EF93FF93E0914F01F0918E
:1007000050018081E0915501F091560182FD1BC09E
:100710009081809158018F5F8F73209159018217CA
:1007200041F0E0915801F0E0E15CFE4F958F80933D
:100730005801FF91EF919F918F912F910F900FBED4
:100740000F901F9018958081F4CF1F920F920FB6D3
:100750000F9211242F933F938F939F93AF93BF9347
:1007600080912B0190912C01A0912D01B0912E012F
:1007700030912A0126E0230F2D3758F50296A11D4E
:10078000B11D20932A0180932B0190932C01A093FB
:100790002D01B0932E0180912F0190913001A091F5
:1007A0003101B09132010196A11DB11D80932F013D
:1007B00090933001A0933101B0933201BF91AF917A
:1007C0009F918F913F912F910F900FBE0F901F908F
:1007D000189529E8230F0396A11DB11DD2CFEFE391
:1007E000F1E01382128288EE93E0A0E0B0E084830F
:1007F0009583A683B7838DE091E09183808385EC18
:1008000090E09587848784EC90E09787868780ECDA
:1008100090E0918B808B81EC90E0938B828B82ECCB
:1008200090E0958B848B86EC90E0978B868B118E75
:10083000128E138E148E63E182E693E00E94790299
:1008400063E084E493E00E94790265E086E293E04D
:100850000E9479026EE088E093E00E94790262E1F2
:100860008AEE92E00E9479026FE08CEC92E00E94A6
:10087000790261E18EEA92E00E9479028EE1E2E67D
:10088000F3E0ACEDB1E001900D928A95E1F78EE1D5
:10089000E4E4F3E0AAEFB1E001900D928A95E1F76C
:1008A0008EE1E6E2F3E0A8E1B2E001900D928A95D4
:1008B000E1F78EE1E8E0F3E0A6E3B2E001900D920B
:1008C0008A95E1F78EE1EAEEF2E0A4E5B2E001906C
:1008D0000D928A95E1F78EE1ECECF2E0A2E7B2E04E
:1008E00001900D928A95E1F78EE1EEEAF2E0A0E93F
:1008F000B2E001900D928A95E1F70895CF93DF93CE
:1009000000D01F92CDB7DEB7789484B5826084BDE5
:1009100084B5816084BD85B5826085BD85B5816003
:1009200085BD80916E00816080936E001092810081
:10093000809181008260809381008091810081603C
:1009400080938100809180008160809380008091FD
:10095000B10084608093B1008091B0008160809389
:10096000B00080917A00846080937A0080917A0050
:10097000826080937A0080917A008E7F80937A00E3
:1009800080917A00806880937A001092C100E09193
:100990004F01F091500182E08083E0914B01F09192
:1009A0004C011082E0914D01F0914E0187E6808369
:1009B00010925701E0915301F091540186E0808339
:1009C000E0915101F0915201808180618083E0913A
:1009D0005101F0915201808188608083E091510142
:1009E000F0915201808180688083E0915101F09103
:1009F000520180818F7D808361E089E00E94E50162
:100A000061E088E00E94E50161E08AE00E94E50182
:100A100060E089E00E94990160E088E00E9499010D
:100A200060E08AE00E94990110923701109238012B
:100A30001092390110923A0110923B0110923C0140
:100A400010923D0188248A94982CA82C8FE0B82E0F
:100A50009EE3292E91E0392E20E0C22E20E0D22EF6
:100A600021E0209301018CED91E09B838A8310E0CB
:100A700000E00983AA81BB8154961D921D921D92AC
:100A80001C9257978D919C9197FDE9C02EE1F894A7
:100A9000AA81BB815996ED91FC915A979281589603
:100AA0008C9158978095892382835C96ED91FC9177
:100AB0005D9791815B968C915B978095892381836B
:100AC0005C96ED91FC915D9792815B968C915B9722
:100AD0008095892382835C96ED91FC915D9781815D
:100AE0005B969C915B97892B81835C96ED91FC9141
:100AF0005D9792815B968C915B9780958923828329
:100B000080E190E00197F1F75C96ED91FC915D97A3
:100B100091815B968C915B978095892381835C960C
:100B2000ED91FC915D9792815B968C915B9780959E
:100B3000892382835996ED91FC915A978281589628
:100B40009C915897892B828378945C966D907C90C9
:100B50005D975B96FC90F3013081EA81FB8184898B
:100B60009589A689B7893F2140855185628573851E
:100B700031110DC084179507A607B70740F40196F9
:100B8000A11DB11D848B958BA68BB78BE4CF481725
:100B900059076A077B0708F462C0F894AA81BB81F1
:100BA0005C96ED91FC915D9782815B969C915B9741
:100BB000892B82835C96ED91FC915D9781815B9698
:100BC0009C915B97892B81835C96ED91FC915D975D
:100BD00082815B969C915B97892B82835C96ED91D9
:100BE000FC915D9791815B968C915B9780958923B1
:100BF00081835C96ED91FC915D9792815B968C91DF
:100C00005B978095892382835996ED91FC915A9741
:100C1000928158968C9158978095892382837894F5
:100C20005C966D907C905D975B963C91F301F080B3
:100C3000EA81FB8184899589A689B789F322408559
:100C4000518562857385FF2029F084179507A607D3
:100C5000B70788F084179507A607B707B0F00F5FAE
:100C60001F4F8A819B814E969B838A830730110593
:100C700009F0FFCEB7C00196A11DB11DEA81FB812D
:100C8000848B958BA68BB78BD1CF215009F0FFCEEB
:100C90000E946D02AA81BB8150964D905D906D902F
:100CA0007C90539764197509860997091C964D9095
:100CB0005D906D907C901F974616570668067906E2
:100CC000C8F554964D905D906D907C905797129614
:100CD0006D917D918D919C911597461657066806EA
:100CE000790609F4BAC0461A570A680A790A0E94B6
:100CF00096072DEC3CEC4CEC5DE30E94FC070E9457
:100D00006007072E000C880B990B461657066806DD
:100D1000790680F4EA81FB8182829382A482B58283
:100D20000E946D02AA81BB8150966D937D938D9335
:100D30009C935397EA81FB8184899589A689B78919
:100D4000428153816481758184179507A607B7078F
:100D500020F482839383A483B583EA81FB8142815B
:100D6000538164817581841B950BA60BB70B843F5F
:100D70009140A105B1050CF472CF70903E01E72CB3
:100D8000F12C772051F0F701EA5CFE4F2081C80179
:100D900001962817190609F462CF61E08AE00E94E3
:100DA0009901F701E95CFE4F89818F5F808373941D
:100DB00070923E010E946D02609333017093340182
:100DC00080933501909336010E94E5021092000154
:100DD0006CE271E080E090E00E943B0260E08AE01B
:100DE0000E94990180913E01873009F040C0E7E3FD
:100DF000F1E0A2E0B1E091918D91981791F11092FC
:100E000001018091010161E0813079F588E00E9463
:100E1000990160ED77E080E090E00E943B0260E0A5
:100E200088E00E94990160E089E00E949901109297
:100E30003701109238011092390110923A01109244
:100E40003B0110923C0110923D010E94E50291E0AD
:100E50009093000110923E0121C0412C512C32018F
:100E600046CF2E163F0639F6CCCF89E0D0CF0E9470
:100E70006D020091330110913401209135013091C0
:100E80003601601B710B820B930B6838734181052F
:100E9000910520F080910001882349F26EE170E015
:100EA00080E090E00E943B02C114D10409F4D8CD47
:100EB0000E94F600882309F4D3CD0E940000D0CD13
:100EC0000E9467076894B1110C94F60708950E9478
:100ED000DB0788F09F5798F0B92F9927B751B0F0EA
:100EE000E1F0660F771F881F991F1AF0BA95C9F7AE
:100EF00014C0B13091F00E94F507B1E008950C9450
:100F0000F507672F782F8827B85F39F0B93FCCF302
:100F1000869577956795B395D9F73EF4909580952A
:100F2000709561957F4F8F4F9F4F0895E89409C04A
:100F300097FB3EF490958095709561957F4F8F4F0C
:100F40009F4F9923A9F0F92F96E9BB279395F69522
:100F5000879577956795B795F111F8CFFAF4BB0FA0
:100F600011F460FF1BC06F5F7F4F8F4F9F4F16C004
:100F7000882311F096E911C0772321F09EE8872F8E
:100F8000762F05C0662371F096E8862F70E060E04A
:100F90002AF09A95660F771F881FDAF7880F9695C3
:100FA000879597F9089557FD9058440F551F59F0AC
:100FB0005F3F71F04795880F97FB991F61F09F3F46
:100FC00079F087950895121613061406551FF2CF6F
:100FD0004695F1DF08C0161617061806991FF1CFBF
:100FE00086957105610508940895E894BB276627E6
:100FF0007727CB0197F908950E940F080C94800879
:101000000E94720838F00E94790820F0952311F0B0
:101010000C9469080C946F0811240C94F6070E9434
:10102000D30770F3959FC1F3950F50E0551F629F52
:10103000F001729FBB27F00DB11D639FAA27F00D31
:10104000B11DAA1F649F6627B00DA11D661F829F58
:101050002227B00DA11D621F739FB00DA11D621F3D
:10106000839FA00D611D221F749F3327A00D611D5A
:10107000231F849F600D211D822F762F6A2F11243C
:101080009F5750409AF0F1F088234AF0EE0FFF1F6F
:10109000BB1F661F771F881F91505040A9F79E3FC6
:1010A000510580F00C9469080C94F6075F3FE4F357
:1010B000983ED4F3869577956795B795F795E7951C
:1010C0009F5FC1F7FE2B880F911D9695879597F925
:1010D000089597F99F6780E870E060E008959FEFBA
:1010E00080EC089500240A941616170618060906BF
:1010F000089500240A94121613061406050608958E
:10110000092E0394000C11F4882352F0BB0F40F415
:10111000BF2B11F460FF04C06F5F7F4F8F4F9F4F55
:101120000895A1E21A2EAA1BBB1BFD010DC0AA1F28
:10113000BB1FEE1FFF1FA217B307E407F50720F040
:10114000A21BB30BE40BF50B661F771F881F991FBB
:101150001A9469F760957095809590959B01AC0104
:10116000BD01CF010895EE0FFF1F0590F491E02D12
:061170000994F894FFCF82
:10117600010105010602030407000000002C018C92
:1011860000B9007901EA00C800DC00536571756595
:0A1196006E63653A000D0A000900BF
:00000001FF
